:10000000080C2500840C2600070C0500000C0600D7
:10001000000C0200030C27000707AF0A080C25009C
:10002000070C05002705200C2C00050C3200680089
:1000300069006A00010C06000000840C0607970C9A
:100040002600000C060005022B0005022F00080CFC
:10005000250007044F0607050F02AB012B07350AE1
:10006000030CEC01050C3200390A32024306EC00A5
:10007000390A0F022B002707420ABB0CCC010306EA
:100080002704470A260C8C000307270500003202CC
:100090004307F2004B0A05022F00020C0E06040D66
:1000A0002706010D05000F02AB012B075D0AEC00CE
:1000B0002706EC0027075F0A5E0A5E0A5F0A0F0246
:1000C0002B002F030F03680369036A038903880168
:1000D0002A06010F30006C0A000005022F00000004
:1000E0006500AB012B077A0AEC002706EC00270716
:1000F0007C0A7B0A7B0A7C0A0F022B00020C0E068C
:10010000040D2706010D05005A0C8C000306AC00F7
:10011000200C8C000307AC0004008E0A00000502CE
:100120002F00070C2707FE0E05000F02AB012B075F
:100130009F0AEC002706EC002707A20AA40AA00ADF
:10014000A10AA20AA30AA40A0F022B00100291011D
:10015000010F2E00100231000706250A0C0A070CB9
:100160000500680069006A006C006D00010C060063
:10017000000006022F00000C06000F07570B010CB1
:100180003000030C3100040C3200060C3300070C65
:100190003400080C3500090C3600350C3700390CDA
:1001A0003800FF0C3900FE0C3A00FD0C3B00F80C47
:1001B0003C00EF0C3D00FC0C3E00840C3F00E00ACC
:1001C000E10A440C2C06D0014C06DE016C06D40179
:1001D0008C06DF01AC06DC01CC06D10126000D0245
:1001E0004507010F2D006504EE0C3E00640C3F0036
:1001F000F90AFA0A0000440C0C06DA012C06D401B4
:100200004C06DD016C06D8018C06DF01AC06DE0170
:10021000CC06D201EC06D90126000D036803690360
:100220006A0389032A06010F010EA801DD0C3E00B6
:10023000700C3F000000440C0C06DB012C06D601BC
:100240004C06DE016C06DF018C06D701AC06DC0132
:10025000CC06D101EC06D0012600070445060705AF
:100260006505EA0C3E00870C3F000400370B380B95
:100270000000440C0C06DB012C06D3014C06DE0109
:100280006C06DF018C06D501AC06DA01CC06D00184
:10029000EC06D901260008022C00FC0C3E00840C60
:1002A0003F00520B530B00000707DF0A0C0A020C39
:1002B0003000050C3100070C3200090C3300120C21
:1002C0003400150C3500340C3600FF0C3700FE0CE2
:1002D0003800FD0C3900F90C3A00EA0C3B00DE0C4A
:1002E0003C00CE0C3D00F80C3E00700C3F00780B3B
:1002F000790B570C2C06D0014C06DE016C06D5019B
:100300008C06DF01AC06DD01CC06D301EC06D8017A
:1003100026000D024507010F2D006504DC0C3E0090
:10032000530C3F00930B940B0000570C0C06D801A4
:100330002C06D3014C06DE016C06DF018C06D601CB
:10034000AC06DC01CC06D201EC06D80126000D0378
:10035000680369036A0389032A06010F010EA801D5
:10036000FB0C3E00820C3F000000570C0C06DE0127
:100370002C06D4014C06DD016C06DF018C06D90188
:10038000AC06DA01CC06D001EC06D7012600070442
:10039000450607056505DA0C3E00890C3F000400A0
:1003A000D10BD20B0000570C0C06D9012C06D20140
:1003B0004C06DB016C06DF018C06DE01AC06D101C8
:1003C000CC06D701260008022C00F80C3E00700C69
:0E03D0003F00EA0BEB0B00000707770B0C0A4F
:0203FE00000AF3
:0804000003000F0000000300DF
:00000001FF
